:100000000C9449050C9466050C9466050C946605E1
:100010000C9466050C9466050C9466050C946605B4
:100020000C9466050C9466050C9466050C946605A4
:100030000C9466050C9466050C9466050C94660594
:100040000C9466050C9466050C9466050C94660584
:100050000C9466050C9466050C9466050C94660574
:100060000C94DF0F0C946605A877A6E0F7435A3589
:1000700085E272978FB71A6287380D67C7BE4F3E09
:100080002076378F68B7A9263F2B10E3307E900E7D
:10009000850A70510386400D4FEB3ECCD18735BDAC
:1000A000F50B5ED0F8F2D5E26C310CADFC21C378D3
:1000B000C106C24C55E64A3448111EDAE71A84A03C
:1000C00096A7E37FAF639CFA235B79C89EBAB2C957
:1000D00022124BB3A1B63249A2E189391066C50795
:1000E0008F54EA91CA3FF919F0D746BC281B61E842
:1000F0002F6AAE9DF64E0914774DDB1F2E7B7CF1E7
:1001000043A300B8138C85B9297588FDD2561C50BD
:100110009741E53B60B5C064EE98D62D25A4AACDE5
:100120007DA883C6ABBE4499263CCE9FBFD3CB7679
:100130007A7E82018A9A801D0EB05CD43862F430D7
:10014000E08E53B70257ACA6520A6D92651724335E
:10015000457274B1B4F75DED2CFF47375A90BBDFA1
:100160002A165995D9C4276773C768FEA5DD6B5F4A
:1001700093D8EC053A8D6EFB3DA96936F394DEEF1A
:10018000156F8B9B080FDC81182004E471CFE92BDD
:10019000425801A0A962D63F85A7B6D4FA156617C2
:1001A00009BD5D14342659729154064FF8B05B7442
:1001B00093998CF245CDEA4EAD104AE5CAEEDFC602
:1001C0006F9F888E02CC08A877946D21B128E439FE
:1001D0007996607181162EE678B9C4469A42AEB718
:1001E0007C43B3221A86C2323D2D9CD229E9639BFF
:1001F000D131385E1E3641BB03182B3EBF6861FC0F
:1002000052C0DEE00A58135A00BE1C900E5312FD75
:10021000E26EBACE2427447F87A3A1D55040E3F9EC
:1002200083F7C7A235C8DB19AB2F1125ED339E55D7
:10023000E148AF7384DA2AAA51EB9D95B2CBE770FF
:1002400080FE4C6504EFC5F1C33AB4F55F2389DD48
:1002500030A58BD3F6DC4D64D7F08FEC56375CA419
:100260000D07768A2C0BB5D8C11FE83BF44B1B4712
:100270006C49677B92CF757E20D97D3C977AD005FB
:100280006B0F1DFB8298578DF36ABCACC9A6FFB8F3
:10029000690C4C4D72075A49338DA2AB463D630D34
:1002A000A097FFF0F5FAC0E9DB62E4E17443DC8675
:1002B000182937F406E2ED6F90481E2D1DEA73945D
:1002C00054DF25F64727D91177C9841C5B5C51811F
:1002D000A6223E2496C88AEC827C09B8454A57BBC0
:1002E0002F50758E61708C6CAFD0FDB41BAEDEFEEE
:1002F0003BB536BD55010E9C41565FB3260383BA0C
:10030000134BCAC50AF860A5B9C7C39832FB12F9E6
:10031000A792AA68F3787E05202102E8BFF2B059BF
:100320008FD2CB876515F11AB230ADEE58A38B662C
:100330001F2CD75D1985A8E6D36BA10C91936A5E3B
:100340000B79E3DD004F3C896E7169A9AC40E599FA
:1003500028C6314E7ACD089E7DEF17FC88D8A46D53
:100360004495D1B7D49BBE2A34642BCF2EEB38CE24
:1003700023E03A3FF77B9F1053BC526716E7807625
:1003800004C4B6C1C27F9ADAD53942149DB10F3583
:10039000D6CCB9DA380CA29C091F06B1B6FD1A6991
:1003A0002330C4DE01D1F45829371C7DD5BFFFBDF1
:1003B000C8C9CF65BE7B7897986708B32657F7FA08
:1003C00040AD8E75A67CDB918B5199D4177A908DB8
:1003D000CE63CB4EA0AB183A5B507F2174C1BBB843
:1003E000B7BA0B359531599A4D04071E5A7613F357
:1003F0007183D08603A83942AA28E6E4D85DD3D019
:100400006E6F96FB5EBC56C25F859BE7AFD23B84A6
:100410006AA753C54449A5F936723D2CD91BA1F5ED
:100420004F939D68474116CA2A4CA387D6E5192EDB
:1004300077156D70C0DFB20046EDC66C4360922D3B
:10044000A922458F3455AEA40A6632E0DC02ACE83E
:10045000208C89624AFEEEC3E33CF17905E9F62778
:1004600033CCF29E11817E80108A829F480DD7B4D2
:10047000FC2FB5C7DD88146B2B54EA1D945CB0EFDC
:100480001224CDEBE1E264733F0E5261253EF80F7A
:100490004BECC00030F602493D106E20C9A62FFE7D
:1004A0002C2B752E4526AB48A980FC04CCD3B5BABD
:1004B000A338317D01D9A77B96B663694EF7DEE09C
:1004C00078CA50AA41916588E42185DA3A27BE1C92
:1004D0003E425E17527F1F89246F8F5C67740E1235
:1004E000878DE934ED73C4F8615B05DF594C97796A
:1004F0008318A45595EBBD53F5F15766469FB2811D
:100500000951862216DD23937629C2D71DD4BF3622
:100510003FEA4B1132B9625460D66D439A0D929CFA
:10052000B0EF586C9D772D70FAF3B30BE2407EF478
:100530008AE58C3C5671D164E1820ACB131590ECAC
:100540000399AF145D0F334A94A5A8351BE36AC61F
:1005500028FF4DE72584AC08AEC5A22AB8370C7A2F
:10056000A0C3CEAD061A9E8BFBD5D0C11ED0B49BC6
:10057000B144F247C768CF72BB4F5AF9DC6BDBD28C
:10058000E87CC8EE98A1E6D839075FFD8E19B73B25
:10059000BCCD7CE38173B211BF6F2098FE7596EFDE
:1005A0006CDA50E109725445BA34805BED3E532C4D
:1005B00087A457F3333F3CB767B4A325604F076B5D
:1005C0001B47150FE40AEAD1327836498D4BD2BC6D
:1005D000A5DC1D0D4DCD9A825FFC9465BEE2F4C989
:1005E0001E44CB9E0C64712663B314E840708A0EDF
:1005F00019426DAC88105CDF41A9ADE5FB74CCD528
:10060000068E5986CE1F3D76E08FB977277BA6D818
:1006100029D3ECB813F7FAC3516ADE4A5AEBC28BFE
:10062000234892CF62A899F8D02E856143C8BDF0C7
:100630000593CA4EF17D30FDC469662F08B152F9A9
:1006400021E67A2BDD3984FFC091D637D47F2D9BEC
:100650005DA13B6EB5C54604F590EE7E831C035646
:10066000B6AA0017013555790B12BB1A31E70228DB
:1006700016C1F6A2DB189C89683897ABC72AD73A0F
:10068000F2C6244CB058A0225E9DD9A7E9AEAF8C2B
:10069000959F28B720D7B030C30919C067D6003C52
:1006A0007EE7E9F4085AF8B82E05A6259E5CD81511
:1006B0000DE1F611546BCD2146665E84AD063829F6
:1006C00044C5A2CEF1AAC1407186B5EFFC36A8CBD5
:1006D0000A48274564A3AF8CB2C69F0789DC17D3AD
:1006E0004979FBFE1DD0B9884352BC01782B7D941B
:1006F000C70EDEA5D59BCCF7617AC274813903ABF6
:1007000096A037BD2D72753FC9D48E6FF98DED62FD
:10071000DB1CDF04AC1B6C144B63D0BFB482EC7BDE
:100720001A5992D21060B63D5FE6806E70C4F23501
:10073000D97CEEE541A45B50DDBB4CF31F9D5D57BA
:10074000555197E358424D9C73BAC877316926AE2C
:10075000EA8ADA22B38756FA930B341633E8E45365
:10076000BEA9B13A3EF5906ACF3B12FD8F9AA747DA
:100770009199EB0F24FF2318854E7F0CE0A1D2D175
:100780002C2A4A024F1E95688B98836D76CA653273
:10079000132FC3829AA4BA8160373435FC80A851E4
:1007A0006567ED305F10D34A272F13B92AD2CCE109
:1007B000EFAEEBBEF4BDCF43B3C58884B7DD39409F
:1007C000CE486D9B72617EE7A14E532E773BE2C906
:1007D00036221B6E73B103B24C87A9D44D0FD815C6
:1007E0006CAA18F649575DFB7A149463A011B09E69
:1007F000DE0546C8EE47DBDC24899C919729E97B1E
:10080000C1071EB8FDFEACC662984FF179E0E86BF7
:100810007856B68D045086CA6F20E6EAE576171C36
:10082000747FBC0D2C85F76696E48B753F4BD938E9
:10083000AF7CDA0B832D3132A2F51D594145BF3C07
:100840001FF8F98AD016256912999D2195AB01A64A
:10085000D7B5C07DFF580E3A92D155E3089FD63EDA
:10086000528EFAA3C702CDDF8F64198CF3A70C5EFA
:100870000A6A09F0935B42C20623EC71ADB4CBBBAC
:100880007028D51A5C33685A004490A5C4263D2BC5
:10089000F25496ADDA1FED33E18169080D0ADB35BC
:1008A000779A64D1FC78AA1BD067A0DDFA6C6371DB
:1008B0000584176A894F667FC65055926FBDE7D28F
:1008C00040728DBBEC06428AE4889D7E7A822713B3
:1008D000411AAFC8A476B4C2FE6D1CD96130B37C96
:1008E000EAF7290FF23B51C1DE5FE52A2F990B5D34
:1008F000A32B4AAB95A5D35856EE283100CC15460C
:10090000CAE686383C65F5E39FD65B094983702DBE
:1009100053A97DE2C4AC8E5EB825F4B957F3F168F3
:1009200047B2A25920CE34795C900E1EBED5222348
:10093000B1C91862162E913E078FD83F933DD49BC4
:10094000DF8521FB117497C7D7DC4C194598E94323
:10095000024BBCC3049C6BF07552A726F6C5BACFF8
:10096000B0B7AE5AA1BF038B80126E0CEBF9C04436
:1009700024EF10F8A88CE87BFF9E2CCD603687B55D
:1009800094A654733A144E011DB6FD37484D39CB29
:10099000E032000000000000000000000000000045
:1009A0000000000000000000000000000000000047
:1009B0000000000000000000000000000000000037
:1009C0000000000000000000000000000000000027
:1009D0000000000000000000000000000000000017
:1009E0000000000000000000000000000000000007
:1009F00000000000000000000000000000000000F7
:100A000000000000000000000000000000000000E6
:100A100000000000000000000000000000000000D6
:100A200000000000000000000000000000000000C6
:100A300000000000000000000000000000000000B6
:100A400000000000000000000000000000000000A6
:100A50000000000000000000000000000000000096
:100A60000000000000000000000000000000000086
:100A70000000000000000000000000000000000076
:100A80000000000000000000000000000000000066
:100A9000000011241FBECFEFD4E0DEBFCDBF11E0B8
:100AA000A0E0B1E0E0EFFAE202C005900D92A43CB4
:100AB000B107D9F714E0A4ECB1E001C01D92A03356
:100AC000B107E1F70E94E10B0C9476150C9400003D
:100AD00081E08093C801089586E291E062E274E0CB
:100AE0004EE050E00E943A15009759F0A2E2B4E0BF
:100AF000E6E2F1E08EE001900D928150E1F70E9474
:100B000002150895FC018091C401882319F46083C3
:100B10000E946C0508950F931F93CF93DF938C0170
:100B2000EB0118861F821C821B821A821982FC012B
:100B30008081833009F4D7C0843020F4823009F0FA
:100B400085C507C0843009F4E4C2853009F07EC54C
:100B500010C180913201F8019181882371F091FFD9
:100B600004C080E490E098878F83F801818180FF42
:100B700027C08F819885806121C090FF04C080E4E8
:100B800090E098878F83F801818181FF05C08F8174
:100B90009885806298878F83F8018181928190FF88
:100BA00005C08F819885806198878F83F801818146
:100BB000928191FF05C08F819885886098878F8387
:100BC00080913301F80191818823B9F094FF02C02C
:100BD00084E68A83F801818185FF02C08CE98A83DB
:100BE000F801818186FF02C08CE98983F801818147
:100BF00087FF25C084E6898322C094FF05C08F81CA
:100C00009885816098878F83F801818185FF05C071
:100C10008F819885906498878F83F801818186FF02
:100C200005C08F819885826098878F83F8018181C4
:100C300087FF05C08F819885906898878F83F8011A
:100C4000818182FF05C08F819885906198878F830D
:100C5000F801818183FF05C08F8198859460988712
:100C60008F83F8018181928192FF05C08F819885E1
:100C7000906298878F83F8018181928193FF05C0EC
:100C80008F819885926098878F83F8018181928106
:100C90008C719C708C519C4031F4109232011092F6
:100CA00033010E946C05F801818192818C729C70E5
:100CB0008C529C4039F481E08093320110923301D0
:100CC0000E946C05F801818192818C749C708C5417
:100CD0009C4009F0BBC481E0809333011092320143
:100CE0000E946C05B3C4F801818180FF04C080E1DB
:100CF00090E098878F83F801818181FF05C08F8103
:100D00009885806498878F83F801818182FF05C070
:100D10008F819885906198878F83F801818183FF07
:100D200005C08F819885946098878F83F8018181B1
:100D300084FF05C08F819885816098878F83F80133
:100D4000818185FF05C08F819885906498878F8306
:100D5000F801818186FF05C08F8198858260988720
:100D60008F83F801818187FF71C48F819885906896
:100D7000CDC1442339F0F801878183FF03C081E0AE
:100D80008093C40180913101823009F47DC08330A9
:100D900030F4882359F0813009F037C134C08330F2
:100DA00009F4B0C0843009F030C1EDC0F80187818A
:100DB00087FF05C08F819885806198878F83F801B0
:100DC000878186FF05C08F819885806498878F838F
:100DD000F801878185FF05C08F8198858860988795
:100DE0008F83F801878184FF05C08F819885806299
:100DF00098878F83F8018781908593FF32C08F8118
:100E0000988584682CC0F801878186FF05C08F8192
:100E10009885806298878F83F801878187FF05C056
:100E20008F819885806498878F83F801878184FFFC
:100E300005C08F819885886098878F83F8018781A6
:100E400085FF05C08F819885806198878F83F80121
:100E50008781908593FF05C08F81988590619887E1
:100E60008F83F8018781908591FF05C08F819885D8
:100E7000906298878F83F8018781908592FFC5C023
:100E80008F8198859260BFC0F801878187FF05C078
:100E90008F819885806198878F83F801878186FF8D
:100EA00005C08F819885806498878F83F80187813A
:100EB00085FF05C08F819885886098878F83F801AA
:100EC000878184FF05C08F819885806298878F8392
:100ED000F8018781908593FF05C08F819885926086
:100EE00098878F83F8018781908591FF05C08F8156
:100EF0009885806898878F83F8018781908592FF15
:100F000084C07EC0F801878187FF05C08F819885E6
:100F1000846098878F83F801878186FF05C08F8161
:100F20009885806198878F83F801878185FF05C048
:100F30008F819885806498878F83F801878184FFEB
:100F400005C08F819885886098878F83F801878195
:100F5000908593FF05C08F819885806498878F83E3
:100F6000F8018781908591FF05C08F819885806801
:100F700098878F83F8018781908592FF46C08F8183
:100F80009885806240C0F801878187FF05C08F8106
:100F90009885806498878F83F801878186FF05C0D4
:100FA0008F819885806298878F83F801878185FF7C
:100FB00005C08F819885806198878F83F80187812C
:100FC00084FF05C08F819885886098878F83F8019A
:100FD0008781908591FF05C08F8198859062988761
:100FE0008F83F8018781908592FF05C08F81988556
:100FF000926098878F83F8018781908593FF05C061
:101000008F819885846098878F83F801878183FF1B
:1010100005C08F819885946098878F83F8018781B8
:10102000908594FF05C08F819885816098878F8314
:10103000F8018781908595FF05C08F819885906420
:1010400098878F83F8018781908597FF05C08F81EE
:101050009885826098878F83F8018781908596FFB5
:1010600005C08F819885906898878F83F80181816A
:10107000898382818A8383818B8384818C83858128
:101080008D8386818E8327813085C901807F907111
:10109000805F904121F481E391E060E009C0C901E3
:1010A000807F9072805F904231F481E391E061E053
:1010B0000E948205CBC2C901807F9078805F9048F2
:1010C00021F481E391E062E0F3CFC901807F907465
:1010D000805F904421F481E391E063E0E9CF207FD9
:1010E0003870205F384009F0B1C2F8018381803C3C
:1010F0002CF481E391E064E00E948205F801848190
:10110000803C0CF0A3C28F819885986098878F836C
:101110009DC2442339F0F801838183FF03C081E03D
:101120008093C401F80123813481C90184719C70CA
:1011300084519C4021F48FE291E060E044C0C901F9
:1011400084729C7084529C4021F48FE291E061E0B3
:101150003AC0C90184749C7084549C4021F48FE28D
:1011600091E062E030C0C90184789C7084589C4052
:1011700021F48FE291E063E026C0C90184709C7184
:1011800084509C4121F48FE291E064E01CC0C901CD
:1011900084709C7284509C4221F48FE291E065E05F
:1011A00012C0C90184709C7484509C4421F48FE265
:1011B00091E066E008C024703C7824503C4829F453
:1011C0008FE291E067E00E9482058091C40188234C
:1011D000A9F4F80123813481C90185709C70855080
:1011E0009C4011F483E006C026703C7026503C40C1
:1011F00029F481E0809330010E946C05F80183811D
:1012000080FF05C08F819885806198878F83F80162
:10121000838181FF05C08F819885806498878F8343
:10122000F801838183FF05C08F819885946098873A
:101230008F8380912F01883021F1F801838184FF11
:1012400005C08F819885816098878F83F80183819D
:1012500085FF05C08F819885906498878F83F801FA
:10126000838186FF05C08F819885826098878F83F0
:10127000F801838187FF05C08F81988590689887E2
:101280008F8380912F01843009F4A2C0853058F4F7
:101290008130E1F1813098F0823009F450C0833020
:1012A00009F039C168C0863009F4DEC0863008F420
:1012B000BFC0873009F412C1883009F02CC1F80191
:1012C000838182FF05C08F819885846898878F838A
:1012D000F8018381948193FF05C08F819885926086
:1012E00098878F83F8018381948192FF05C08F8155
:1012F0009885906298878F83F801838194818474A4
:10130000907F8454904F09F006C100C1F801838199
:1013100082FF05C08F819885906298878F83F8013E
:101320008381948193FF05C08F819885926098870F
:101330008F83F8018381948192FFEDC0CBC0F801C7
:10134000838182FF05C08F819885906298878F8303
:10135000F8018381948193FF05C08F819885926005
:1013600098878F83F8018381948192FFD4C08F8105
:1013700098859064CEC0F8018381948192FF05C066
:101380008F819885906498878F83F80183819481F9
:1013900093FF05C08F819885846898878F83F801B3
:1013A000838182FF05C08F819885926298878F83A1
:1013B000F8018381948196FF05C08F8198858062B2
:1013C00098878F83F8018381948195FFA4C02CC0F6
:1013D000F8018381948192FF05C08F81988584688C
:1013E00098878F83F8018381948193FF05C08F8153
:1013F0009885926098878F83F801838182FF05C06A
:101400008F819885906298878F83F801838194817A
:1014100096FF05C08F819885806298878F83F80139
:101420008381948197FF77C08F819885886071C090
:10143000F8018381948192FF05C08F819885906225
:1014400098878F83F8018381948193FF05C08F81F2
:101450009885926098878F83F801838182FF5BC0B3
:101460008F819885906255C0F8018381948192FFA5
:1014700005C08F819885906898878F83F801838154
:10148000948193FF05C08F819885926098878F83A0
:10149000F801838182FF05C08F81988590629887CB
:1014A0008F83F8018381948195FF05C08F81988592
:1014B000886098878F83F8018381948196FF05C0A7
:1014C0008F819885806298878F83F80183819481CA
:1014D00097FF21C08F81988584681BC0F8018381A4
:1014E000948192FF05C08F819885846898878F8347
:1014F000F8018381948193FF05C08F819885926064
:1015000098878F83F801838182FF05C08F8198853A
:10151000886298878F8380912F01883019F18430F9
:1015200009F46CC0863009F469C0F80183819481A4
:1015300094FF02C084E68C83F8018381948195FF37
:1015400002C08CE98C83F8018381948196FF02C0EC
:101550008CE98B83F8018381948197FF4FC084E6E7
:101560008B834CC0F801838194812091C50194FF45
:1015700009C020FD0AC08091C6018F5F8093C6011B
:10158000216001C02E7F2093C501F80183819481E1
:101590002091C50195FF09C021FD0AC08091C601B7
:1015A00081508093C601226001C02D7F2093C50128
:1015B000F801838194812091C50196FF09C022FD25
:1015C0000AC08091C7018F5F8093C701246001C06A
:1015D0002B7F2093C501F801838194812091C5015F
:1015E00097FF09C023FD0AC08091C70181508093F5
:1015F000C701286001C0277F2093C50180912F017A
:10160000883031F0F8018181898382818A831EC00C
:10161000F801838184FF03C08091C6018A83F801A9
:10162000838185FF04C08091C60181958A83F8017A
:10163000838186FF03C08091C7018983F80183817C
:1016400087FF04C08091C70181958983DF91CF9185
:101650001F910F91089587FD05C00E947211982F68
:10166000905E05C081950E94721190E2981B892FAF
:101670000895FF920F931F93CF93DF93EC018B019B
:1016800041305105B1F480912F01883061F06091B3
:101690003001898170E00E942B0BF82E609130019F
:1016A0008A8170E012C0F98080E2F80E7A81705E63
:1016B00029C04230510569F4898162E070E00E94DE
:1016C0002B0BF82E8A8162E070E00E942B0B782FA2
:1016D00019C08981992787FD909580589F4F9595CE
:1016E0008795959587953FE3F32EF8228A81992770
:1016F00087FD909580589F4F9595879595958795EF
:10170000782F7F734C81552747FD509540585F4F88
:1017100083E0559547958A95E1F74F716D81659501
:1017200065956595EE818B81992787FD9095805809
:101730009F4FB3E095958795BA95E1F78F71282F64
:1017400030E0A3E0220F331FAA95E1F7822F807CBF
:101750008F29D8018C93220F331F220F331F822F22
:10176000807C872B11968C93119770E0CB01887148
:101770009070880F991F880F991F482B220F331FD5
:10178000220F331F422B12964C93129785E0660F5F
:10179000771F8A95E1F7E695E695E695E62B139691
:1017A000EC9313978885809514968C9314978F816A
:1017B000809515968C93DF91CF911F910F91FF909B
:1017C00008952F923F924F925F926F927F928F92E5
:1017D0009F92AF92BF92CF92DF92EF92FF920F93C0
:1017E0001F93DF93CF93CDB7DEB76B970FB6F89407
:1017F000DEBF0FBECDBF87E088B983EC87B915B8CF
:101800009FEF94B980E18BB99AB90E940B15882398
:1018100019F00E946C0509C0A6E2B1E0E2E2F4E032
:101820008EE001900D928150E1F70E941D113C0164
:101830000E949B118A8F9B8F0E94B814898FA92EBA
:101840008E01005F1F4F80E090E0B80140E00E94F1
:101850008B05C8018E010F5F1F4FB80140E050E0BB
:101860000E94390B80E091E0B80146E051E028E6A3
:1018700035E00E94FC0C7894CC24DD2410E0BB24DD
:10188000EE24FF2400E077E0872E912C8C0E9D1E25
:1018900060E1262E312C2C0E3D1E2E010894411C99
:1018A000511C83B78E6083BF83B7816083BF8895E7
:1018B00083B78E7F83BF8091C8018823E1F31092A4
:1018C000C80189E89BE10197F1F7112321F011305C
:1018D00009F045C028C01092C4010E9497138130BE
:1018E000910551F0029781F4898D9A2D9C0169012F
:1018F00011E052E0B52E15C08A8D9B8D9C016901C7
:1019000011E0BB24B3940DC0D3011296ED91FC916C
:1019100013970995D3011696ED91FC911797C40181
:10192000099501E01DC0D6011296ED91FC91139727
:101930000995882341F00894E11CF11CBBE0EB16EB
:10194000F1046CF40DC0D6011696ED91FC91179739
:10195000C401099501110F5FEE24FF2401C010E0BE
:10196000C401B101402F0E948B0503300CF000E050
:10197000C101B2014B2D50E00E94390BC2010E94FF
:10198000F30C8FCF1092ED021092EC02880F80932F
:10199000BA0085E48093BC0078940895882311F000
:1019A00085EC01C085E88093BC000895282F30E0C5
:1019B00070E088E090E0861B970BA90102C0440FFD
:1019C000551F8A95E2F7CA0102C0359527956A9599
:1019D000E2F7822B0895863028F4E091CA01F09155
:1019E000CB0109950895ACEEB1E0FC0186E00190D1
:1019F0000D928150E1F708950F931F93182F092F2F
:101A00003093CB012093CA01ACEEB1E0FB0186E03C
:101A100001900D928150E1F71092DC02812F902FFE
:101A20009C01D9012AEF30E08D91F901E451FE4F7C
:101A300080832F5F3F4F81E020303807A9F7DA011C
:101A400020E230E08D91F901E451FE4F80832F5F59
:101A50003F4F20343105B1F7459844981092ED027C
:101A60001092EC0284EA8093BA0085E48093BC0073
:101A700078941F910F9108952F923F924F925F9209
:101A80006F927F928F929F92AF92BF92CF92DF928E
:101A9000EF92FF920F931F93DF93CF93CDB7DEB7F3
:101AA00068970FB6F894DEBF0FBECDBF48E6642E30
:101AB00040E0742E882437E0232E312C2C0E3D1E5E
:101AC00028E0422E512CCBC084918D933196A215E3
:101AD000B305D1F780E090E0FC01E453FE4FE081D4
:101AE000F0E0EE56FF4FE491ADE0B0E0AC0FBD1F6B
:101AF000A80FB91FEC9301968A30910569F7AA885F
:101B0000CF8429812A2530E04C2D477050E09E88F3
:101B1000B988C201841B950BB90102C0660F771FFB
:101B20008A95E2F7CB0102C0359527954A95E2F7F1
:101B3000822B89198B258F83EE84DD842A812E25C3
:101B400030E04D2D477050E0AC89C201841B950BED
:101B5000F90102C0EE0FFF1F8A95E2F7CF0102C024
:101B6000359527954A95E2F7822B8A198A27888727
:101B7000EB892B812E2730E00D89077010E0B20130
:101B8000601B710BC901062E02C0880F991F0A94B1
:101B9000E2F7002E02C0359527950A94E2F7822BD2
:101BA0008C198D2589872C812B2530E04A2F477091
:101BB000842F90E0988F8F8BD888C2014F89588DE1
:101BC000841B950BA90102C0440F551F8A95E2F7AB
:101BD000CA010F8802C0359527950A94E2F7822B37
:101BE0008D198C258A878D81E826FF24E770F0E027
:101BF000C2018E1B9F0B970102C0220F331F8A95D3
:101C0000E2F7C90102C0F594E794EA95E2F78E295C
:101C10008D198B258B878E81A827B0E0AD0102C07E
:101C2000440F551F6A95E2F7BA0102C0B595A79512
:101C30000A95E2F76A2B6A1969256C87C10166ED7E
:101C400071E046E050E00E943A15009779F08394E5
:101C500066E070E0660E771E77E0871621F0DE0101
:101C60001196F30131CF1092C9013DC1282D30E00A
:101C70002F5F3F4F522F44278091DA01FA01E80F7E
:101C8000F11DEE56FF4F94912F5F3F4F322F2227C9
:101C90008091CF01F901E80FF11DEE56FF4FE4915D
:101CA000E927E093DC018091D801FA01E80FF11DEA
:101CB000EE56FF4F94918091D101F901E80FF11D8B
:101CC000EE56FF4FE491E927E093DD018091DB01BF
:101CD000FA01E80FF11DEE56FF4F94918091D30168
:101CE000F901E80FF11DEE56FF4FE491E927E0936B
:101CF000DE018091D601FA01E80FF11DEE56FF4F8B
:101D000094918091CE01F901E80FF11DEE56FF4F3D
:101D1000E491E927E093DF018091D701FA01E80F10
:101D2000F11DEE56FF4F94918091D001F901E80F1B
:101D3000F11DEE56FF4FE491E927E093E001809119
:101D4000D901FA01E80FF11DEE56FF4F94918091F1
:101D5000D501F901E80FF11DEE56FF4FE491E92797
:101D6000E093E1018091CC01FA01E80FF11DEE56FC
:101D7000FF4F94918091D201F901E80FF11DEE56C9
:101D8000FF4FE491E927E093E2018091CD01FA0150
:101D9000E80FF11DEE56FF4F94918091D401F901A7
:101DA000E80FF11DEE56FF4FE491E927E093E301C0
:101DB0008091D601FA01E80FF11DEE56FF4F949184
:101DC0008091CD01F901E80FF11DEE56FF4FE4912E
:101DD000E927E093E4018091DB01FA01E80FF11DAE
:101DE000EE56FF4F94918091D001F901E80FF11D5B
:101DF000EE56FF4FE491E927E093E5018091D90188
:101E0000FA01E80FF11DEE56FF4F94918091CC013D
:101E1000F901E80FF11DEE56FF4FE491E927E09339
:101E2000E6018091D801FA01E80FF11DEE56FF4F4F
:101E300094918091D501F901E80FF11DEE56FF4F05
:101E4000E491E927E093E7018091DA01FA01E80FD4
:101E5000F11DEE56FF4F94918091D301F901E80FE7
:101E6000F11DEE56FF4FE491E927E093E8018091E0
:101E7000D701FA01E80FF11DEE56FF4F94918091C2
:101E8000D401F901E80FF11DEE56FF4FE491E92767
:101E9000E093E9018091CF01FA01E80FF11DEE56C0
:101EA000FF4F94918091D101F901E80FF11DEE5699
:101EB000FF4FE491E927E093EA018091CE01480FBA
:101EC000511D4E565F4FFA0194918091D201280F17
:101ED000311D2E563F4FF901849189278093EB01E4
:101EE00081E08093C90168960FB6F894DEBF0FBEFB
:101EF000CDBFCF91DF911F910F91FF90EF90DF90B9
:101F0000CF90BF90AF909F908F907F906F905F9099
:101F10004F903F902F900895982F80548630A0F4D2
:101F200020E430E049E450E0FA01E21BF30BD90170
:101F3000A451BE4F8C91E453FE4F80832F5F3F4FDF
:101F40002634310589F70895892F86548630C8F4E0
:101F5000809132028093CF01809133028093CE0131
:101F6000809134028093CD01809135028093CC0121
:101F7000809136028093DB01809137028093DA01F1
:101F80000895892F8C548430C8F48091380280934E
:101F9000D901809139028093D80180913A028093CF
:101FA000D70180913B028093D601892F90E0860F64
:101FB000911D8035910511F40E943C0D08951F92EA
:101FC0000F920FB60F9211242F933F934F935F936D
:101FD0006F937F938F939F93AF93BF93EF93FF93F1
:101FE0008091B90090E0887F907080399105E9F187
:101FF00081399105D4F480379105A1F1813791059C
:1020000044F48036910571F18836910509F0C2C01B
:1020100029C08038910549F18838910509F4BAC082
:102020008837910509F0B6C01DC0803B910509F4C1
:1020300070C0813B91054CF4803A910509F45DC074
:10204000883A910509F0A6C064C0803C910509F466
:102050009FC0883C910509F49BC0883B910509F01D
:1020600099C05FC01092EE0293C08091EE02882367
:10207000B9F12091BB008091EC029091ED02803F7C
:10208000910531F4253511F02A3A11F41092C90165
:102090008091C9018823E1F0A091EC02B091ED029A
:1020A000E091EC02F091ED02E770F070EC51FE4F20
:1020B0008081E091EC02F091ED02E770F070E45263
:1020C000FE4F90818227890FA451BE4F8C9352C03E
:1020D000E091EC02F091ED02E451FE4F20834AC002
:1020E0008091BB0090E09093ED028093EC0281E040
:1020F0008093EE021092EF024BC08091EC0290911F
:10210000ED022091EF026091EF02821B0E948C0F82
:102110003FC08091EC029091ED020E94EB0C109276
:10212000EF028091C9018823E1F0E091EC02F09187
:10213000ED02E451FE4F8081E091EC02F091ED025E
:10214000E770F070E452FE4F2081E091EC02F091D4
:10215000ED02E770F070EC51FE4F9081821B8927F1
:1021600007C0E091EC02F091ED02E451FE4F808156
:102170008093BB008091EC029091ED0201969093C8
:10218000ED028093EC028091EF028F5F8093EF026B
:1021900085EC01C085E88093BC00FF91EF91BF9171
:1021A000AF919F918F917F916F915F914F913F91EF
:1021B0002F910F900FBE0F901F901895419A80E3BA
:1021C0008A95F1F7419880E090E030E048E1242FD3
:1021D0002A95F1F740983695329B3068242F2A953E
:1021E000F1F7409A01968830910589F73093F10212
:1021F00080E090E048E1242F2A95F1F74098369549
:10220000329B3068242F2A95F1F7409A0196883046
:10221000910589F73093F20280E008951F931FB76C
:10222000F894399A389A3A98429A409A41980E947A
:10223000DE101FBF80E01F91089584E391E00895B0
:10224000FC01009719F12091F1028091F202482FD0
:1022500050E0CA01807F9070803F910521F481E0B9
:102260008093F00202C01092F0028091F002882365
:1022700021F083E08083218309C082E08083942F52
:10228000882730E0822B932B928381838091F10207
:102290009091F2029093F4028093F302089581EFFB
:1022A00092E063EF72E042E050E00E943A15089538
:1022B0008823B9F021E0A82FBB27A7FDB0950BC05C
:1022C000E60FF71F808190E0A817B9071CF4822F52
:1022D000815008952F5FE22FF0E0E417F50784F3B3
:1022E0008FE10895623061F0633019F060E471E0CD
:1022F00002C060E671E040E250E00E94581108958B
:1023000060E871E040E250E00E9458110895209189
:10231000AC01253079F0222369F0892B31F023308C
:1023200049F082E08093AC010895213019F084E0F7
:102330008093AC01089580EA91E00895CF92DF92F6
:10234000EF92FF921F93DF93CF930F92CDB7DEB73B
:1023500085E08093AC0110E08CE2C82E81E0D82E9D
:102360007E010894E11CF11C12C0F6013197F1F7CF
:102370000197D9F71982C70161E070E00E94E41269
:10238000489741F01F5F1F3011F480E004C08CE2D9
:1023900091E0EBCF81E00F90CF91DF911F91FF9003
:1023A000EF90DF90CF900895009741F0DC01E5EFCA
:1023B000F2E089E001900D928150E1F7AEEFB2E0DA
:1023C000E5EFF2E089E001900D928150E1F7089588
:1023D00085EF92E06EEF72E049E050E00E943A151E
:1023E00008951F93DF93CF93CDB7DEB7A6970FB6AF
:1023F000F894DEBF0FBECDBF1982CE01019661E019
:1024000070E00E94E412883119F01092AC016DC0A6
:1024100080913503882331F08091AC01853011F42F
:102420001092AC0180913503882319F485E08093E4
:10243000AC018091AC018230E9F08430A1F18823B5
:1024400009F049C083E0898380E88A8381E08B8337
:10245000CE01049660E870E042E250E00E94471529
:10246000CE01019663E270E00E94E412882399F1A4
:1024700084E02FC013E0198380EC8A838BE18B8387
:10248000CE01049661E070E040E250E00E94471502
:10249000CE01019663E270E00E94E4128823D9F035
:1024A0001093AC0118C083E0898380EC8A838BE1B0
:1024B0008B8380E2FE013496DF011D928A95E9F755
:1024C000CE01019663E270E00E94E412882319F0C5
:1024D00081E08093AC0181E08983CE01019661E0C7
:1024E00070E00E94E412803211F08FEF5AC084E055
:1024F0008093F50220E030E040E050E061E070E0E1
:10250000F901E25EFC4F8081882349F0CB01022E65
:1025100002C0880F991F0A94E2F7482B592B2F5FAE
:102520003F4F2031310561F75093F9024093F80293
:1025300019821A8240E020E030E060E870E0F901A2
:10254000E25DFC4F8081882339F0CB01022E02C06E
:10255000959587950A94E2F7482B2F5F3F4F2830D7
:10256000310569F749834A8120E030E060E870E096
:10257000F901EA5CFC4F8081882339F0CB01022EFF
:1025800002C0959587950A94E2F7482B2F5F3F4F3D
:102590002830310569F789818093F6024093F7026C
:1025A00080E0A6960FB6F894DEBF0FBECDBFCF91E8
:1025B000DF911F9108950E94F11180E008953B98EA
:1025C0004398249A2C980895EF92FF920F931F93AB
:1025D000CF93DF937C01662309F456C070E020E0BE
:1025E00030E0E0E0F0E011C088818423FD01E25E8C
:1025F000FC4F808311964695A017B107A9F72F5F6E
:102600003F4F2617370754F4FD01DF0140E8E7018B
:10261000C20FD31F8F01085F1F4FE6CFEEE1F3E03B
:10262000CF93DF93EF93FF930191002311F069F4AF
:102630001BC000003B9A1DE014D03B980000000036
:1026400000000000119781F70FC03B9A12E00000D4
:1026500008D03B9819E005D000000000119721F741
:1026600003C01A95F1F7089500000000FF91EF9163
:10267000DF91CF913B9A12E00000F3DF3B980FEF20
:102680000A9511F0339BFCCFEEE1F3E0EF93FF935B
:10269000112700270395A1F03399FCCF08C00BE464
:1026A000039572F03399FCCF139551F001930BE42D
:1026B000039532F0339BFCCF139511F00193EFCFCC
:1026C000FF91EF91612F70E06115710531F110FFFD
:1026D00024C040E050E020E030E00CC08081F901EF
:1026E000E35EFC4F9081E0E0891708F4E1E0EC93B1
:1026F0004F5F5F4FDA01A25EBC4FF901E25EFC4F13
:102700002E5F3F4F411750F384E18A95F1F79B010B
:10271000215030403595279502C020E030E0C901B6
:10272000DF91CF911F910F91FF90EF900895DF936C
:10273000CF930F92CDB7DEB71982CE01019661E03B
:1027400070E00E94E412009719F420E030E026C007
:10275000489711F580912203882311F098E001C079
:1027600090E0809123038111946080912403811172
:10277000926080912503811191609A3028F49830FD
:1027800028F4953049F405C09B3031F422E030E064
:1027900005C021E030E002C023E030E0C9010F9025
:1027A000CF91DF91089585E08093080320E030E029
:1027B00040E050E061E070E0F901E25EFC4F8081B2
:1027C000882349F0CB01022E02C0880F991F0A947A
:1027D000E2F7482B592B2F5F3F4F2031310561F72E
:1027E0005093100340930F0320E030E070E040E886
:1027F00050E0F901E25DFC4F8081882339F0CA0185
:10280000022E02C0959587950A94E2F7782B2F5FE8
:102810003F4F2830310569F720E030E060E040E8C4
:1028200050E0F901EA5CFC4F8081882339F0CA014D
:10283000022E02C0959587950A94E2F7682B2F5FC8
:102840003F4F2830310569F720E030E040E0A0E854
:10285000B0E0F901E25CFC4F8081882339F0CD01C2
:10286000022E02C0959587950A94E2F7482B2F5FB8
:102870003F4F2830310569F740930B0320E030E0EB
:1028800050E0A0E8B0E0F901EA5BFC4F80818823CA
:1028900039F0CD01022E02C0959587950A94E2F792
:1028A000582B2F5F3F4F2830310569F78091070380
:1028B0008823D1F080911A03781B709309038091CB
:1028C0001B03681B60930A0380911C03481B409301
:1028D0000B0380911D03581B50930C0340E020E034
:1028E00030E060E870E014C070931A0360931B033B
:1028F00040931C0350931D031092090310920A0386
:1029000010920B0310920C0381E080930703E6CF33
:10291000F901E25BFC4F8081882339F0CB01022E64
:1029200002C0959587950A94E2F7482B2F5F3F4F99
:102930002830310569F740930D0340E020E030E096
:1029400060E870E0F901EA5AFC4F8081882339F091
:10295000CB01022E02C0959587950A94E2F7482B89
:102960002F5F3F4F2830310569F740930E030895DC
:102970008DEA91E00895009741F0DC01E8E0F3E092
:1029800089E001900D928150E1F7089588E093E08D
:1029900061E173E049E050E00E943A150895DF9349
:1029A000CF93CDB7DEB728970FB6F894DEBF0FBE32
:1029B000CDBF80E4898383E08A831B82CE010196A8
:1029C00063E070E00E94E412803411F081E003C003
:1029D0000E94D31380E028960FB6F894DEBF0FBE96
:1029E000CDBFCF91DF910895109207030E94CF14BD
:1029F00090E0882309F491E0892F08950E94CF1474
:102A000080E0089582E294E060E070E04EE050E003
:102A10000E945E150895CF93DF93C2E2D4E0CE0109
:102A200060E070E04EE050E00E944E15CE0169EB90
:102A300071E049E050E00E943A15009711F480E0FF
:102A400016C08EE0FE0111928A95E9F7DE01E9EBEE
:102A5000F1E089E001900D928150E1F782E294E08B
:102A600060E070E04EE050E00E945E1581E0DF9192
:102A7000CF910895FB01DC0104C08D910190801974
:102A800021F441505040C8F7881B990B0895DC0190
:102A900001C06D9341505040E0F70895DC01CB0137
:102AA000FC01F999FECF06C0F2BDE1BDF89A31965E
:102AB00000B40D9241505040B8F70895DC01CB01AD
:102AC00003C02D910E94691541505040D0F70895E0
:102AD000262FF999FECF1FBA92BD81BD20BD0FB63A
:102AE000F894FA9AF99A0FBE01960895F894FFCFD8
:102AF0000000A4200101E02080E02080E02080E0B0
:102B0000208000000000E02080E02080E02080E0C5
:102B10002080000000000000000000000000000015
:102B2000030000000E11DE104F1120110000000004
:102B300000010203060C12161F2832383C404345A0
:102B4000464748494A00000000000000000000001D
:102B5000000102030406080A0C0E10121920262C8C
:102B6000343C3D3E3F404142434445464748494A44
:102B7000000104070B0F13171B1F252B32393F458C
:102B8000494D505356595C5E6061626364000000B9
:102B9000DB12F111E811D41187119E1105FE14CF3B
:102BA00014C614BB140000F414455854454E4D4F40
:042BB0005445000088
:00000001FF
